:100A9E00313131310D0A0030313233343536373899
:060AAE00392E2D4D000061
:1008A90011212050656368696E20536369656E6321
:0308B900652000B7
:100A3D007C64EF4E60131CEC60087D0A1DED60F6C2
:090A4D0080FAEF1F70EC1E80E935
:010A5600227D
:100A8800758921759850758DFD858D8BE4F587D214
:060A9800AFD2ACD28E22A9
:07000300AE071FEE70FA22A8
:0E0B7200C2ACC2998F993099FDC299D2AC22C3
:100A700012037BFF6011120B727F051200037401D9
:080A800029F9E43AFA80E922A9
:10085300E4F50FF510120ACA120ADE120A88750BA4
:100863000A7F011209867532008F337F08120986C9
:100873007534008F357542007543787F05120986FC
:100883007542008F43E5334534F53AE535F53B12C0
:100893000B367BFF7A0A799E120A7012040912073B
:0608A300EC120B8580E958
:100AF20075A0FFC287D286D285AFA0C285EF20E75C
:010B0200F6FC
:010B030022CF
:100B1600AE07120AF2C287C2868EA0D285C285228D
:100B2600AE07120AF2D287C2868EA0D285C285226D
:100B0400ED7004AC078004EF2440FCEC4480FF0249
:020B14000B16BE
:100A0400AE07AC0353050153060FED6003430640E4
:0D0A1400430680AF06120B16AF04020B263E
:100938008B118A128913120B04AB11AA12A9131274
:10094800037B60130513E5137002051214F91203F3
:080958007BFF120B2680E22256
:100ACA007F38120B167F0C120B167F06120B167F3D
:040ADA0001020B16F4
:1008BC00010800010D00010E00010C00010B00C12C
:0708CC0083C1840209000052
:1009A800E4FDFCC3ED9FEC9E5015E4FBFA0BBB0085
:0F09B800010ABA07F8BBD0F50DBD00010C80E4B1
:0109C700220D
:0F0B3600750D03850B0CC286D287D284C285222F
:0F0B4500750D03750C04D286C287C284D2852237
:0B0B9B00E4F50D750C04D284C2852225
:0B0BA600E4F50C750D04C286D2872216
:1009C800300418E508D3950D5004D2B58002C2B59D
:0E09D800E508C394144006E4F50822C2B522D7
:1009E600300318E50ED3950C5004D2B48002C2B47D
:0E09F600E50EC394144006E4F50E22C2B422AE
:03001B00020A21B5
:100A2100C0E0C0D0758DFC758B18050AE50A70020F
:0C0A31000509050E1209E6D0D0D0E03215
:050B8000120B85D2817B
:080B85007F017E02DEFEDFFAB3
:010B8D002245
:0F0B5400D280120B80C280120B85C281020B85EA
:0A0BB100C280120B80D280020B8577
:0208F700AD074B
:1008F900E4FBFAEDC4131313540124FF9280ED2590
:10090900E0FD120B80C281120B850BBB08E5D2807A
:10091900120B85D28130800F0AEAD394C840F6C2FF
:0E09290081120B857F0022C281120B857F0197
:01093700229D
:10096000E4FDFCD280120B85D281120B85EC25E0D0
:10097000FCA280E4334204120B85C281120B850D68
:05098000BD08E5AF0415
:01098500224F
:100A5700AC05A907120B547FA01208F7AF011208C3
:090A6700F7AF041208F7020BB10D
:02098600AC07BC
:10098800120B547FA01208F7AF041208F7120B5489
:0F0998007FA11208F7120960AD07120BB1AF056E
:0109A700222D
:100AB40053706565643A004B4D2F68004C3A004D05
:060AC40000513A002E0073
:1008D300024200070249000002440000014D0002E9
:1008E3003C0000024B0000C101C100C102014600EF
:0308F300015200AF
:040B63007FE87E03A6
:0B0B6700EF1FAC0670011E4C70F62260
:100ADE00758921758C3C758AB0D2A9D28CD2AFD2D1
:040AEE00AAD28A22DC
:100409003001030205F27F0A1209867549008F4AF5
:10041900D3E5439407E5429400400A7F0512098613
:100429007542008F43E4FDFF120B047BFF7A0A79C2
:10043900B4E4FDFF120938AE49AF4A7C007D64126D
:1004490003A67C007D0A1203A6ED2430FF120B26B9
:10045900AE49AF4A7C007D0A1203A67C007D0A12D0
:1004690003A6ED2430FF120B26AE49AF4A7C007D6E
:100479000A1203A6ED2430FF120B267BFF7A0A79B4
:10048900BBE4FD7F0A1209387BFF7A0A79C07D0136
:10049900E4FF120938AE3AAF3B7C277D101203A660
:1004A9007C007D0A1203A6ED2430FF120B26AE3A1A
:1004B900AF3B7C037DE81203A67C007D0A1203A6EC
:1004C900ED2430FF120B26AE3AAF3B7C007D64125F
:1004D90003A67C007D0A1203A6ED2430FF120B2629
:1004E900AE3AAF3B7C007D0A1203A67C007D0A125E
:1004F90003A6ED2430FF120B26AE3AAF3B7C007DFC
:100509000A1203A6ED2430FF120B267BFF7A0A7923
:10051900C37D017F07120938D3E53B94E8E53A9496
:10052900034031E53B2418FDE53A34FCFCE41202B2
:10053900C17B6F7A127903783B120116E4FBFA79D1
:10054900E078401200251202FA8E428F43AD437FB4
:1005590005120A57AE42AF437C007D0A1203948EFE
:10056900428F437BFF7A0A79C57D017F09120938D9
:10057900AE42AF437C037DE81203A67C007D0A12DC
:1005890003A6ED2430FF120B26AE42AF437C007D5B
:10059900641203A67C007D0A1203A6ED2430FF1223
:1005A9000B26AE42AF437C007D0A1203A67C007D78
:1005B9000A1203A6ED2430FF120B267BFF7A0A7973
:1005C900C87D017F0E120938AE42AF437C007D0A17
:1005D9001203A6ED2430FF120B26AE42AF437C0076
:0A05E9007D0A1203A68E428F432202
:1007EC0020B43B120B6320B4327F0A120986754980
:1007FC00008F4A7F01120986753E008F3F7F0812D9
:10080C0009867540008F41E53F4540F53AE541F5D5
:10081C003B7F051209867542008F4330B4FD20B52D
:10082C000B120B6320B502D20230B5FD20B21712A9
:10083C000B6320B20EE50BC394144005750B0180BD
:07084C0002050B30B2FD2292
:03000B000205F3F8
:1005F300C0E0C0F0C083C082C0D075D000C000C0CE
:1006030001C002C003C004C005C006C007758C3C0E
:10061300758AB0054DE54D75F00584E5F07002B2BD
:1006230000E54D75F00A84E5F06003020745E546F1
:1006330060021546E55260021552754D00C2AA8547
:10064300444B85454C754400754500D2AAAE4BAF6B
:100653004C7C007D06120394AC06AD07E41202C184
:10066300E4FBFAF9783F120116C004C005C006C0C6
:1006730007AC3CAD3DE41202C1E4FBFAF9783F124A
:100683000116D003D002D001D0001200251202FAC5
:100693008E3C8F3D300203020722AC3CAD3DE41299
:1006A30002C17B9A7A997919783E1201161202FADD
:1006B3008E498F4AAD4A7F0A120A57AC4BAD4CE4C0
:1006C3001202C1E4FBFA79207840120116E4FBFA26
:1006D30079A0784112021FC004C005C006C007AC50
:1006E3003AAD3BE41202C1D003D002D001D00012D4
:1006F30000251202FA8E3A8F3B853A47853B4875AF
:100703005000853B51AD517F08120A57120B63E528
:1007130047F54F754E00AD4F7F01120A5780237581
:100723003A00753B00754200754307AD3B7F0112EC
:100733000A57AD3B7F08120A57AD437F05120A578C
:10074300C202D007D006D005D004D003D002D00116
:0D075300D000D0D0D082D083D0F0D0E032E2
:03001300020B8E4F
:0D0B8E00C0E00545E54570020544D0E032A9
:10001E00020366E86480F8E933E83360110460F0A7
:10002E00ED33EC337009E8FCE9FDEAFEEBFF220448
:10003E0060DED3EB9FEA9EE99DE8C2E78CF0C2F743
:10004E0095F0400CE8CCF8E9CDF9EACEFAEBCFFB0F
:10005E0012033185D0F05804700320D5B3E8047034
:10006E00075002B2D502037092D5EC0460F7E4CCCF
:10007E00C0E0C398F8603B94186008400DD0E0FBD8
:10008E00020348E4FBFAC9FC8028E830E406E4C920
:10009E00FBE4CAFCE830E305E4C9CACBFCE854072C
:1000AE006010F8C3E913F9EA13FAEB13FBEC13FC37
:1000BE00D8F130F52FC3E49CFCEF9BFFEE9AFEEDDA
:1000CE0099FDD0E0FBEF4E4D4C701222DB03020384
:1000DE006DEC2CFCEF33FFEE33FEED33FDED30E730
:1000EE00EB020348EF2BFFEE3AFEED39FDD0E0FBBD
:1000FE0050130BBB0003020370ED13FDEE13FEEF66
:08010E0013FFEC13FC0203488F
:10011600EC4D6011E8497017ED33EC3304600DE4E3
:10012600FCFFFEFD22E933E8330470F80203661291
:10013600033158046009E4CC248150062850090292
:10014600037028400302036DC0E0EB4A7044B98097
:1001560006D0E0FB02035CEF4E701CBD8008EBFF8F
:10016600EAFEE9FD80EBE98DF0A4FEE5F00201FF71
:10017600E9CDF9EAFEEBFFEF89F0A4FCE5F0CE89C4
:10018600F0A42EFFE435F0CD89F0A42DFEE435F081
:100196008067EF4E7005BD80D780C3EF8BF0A4ACAF
:1001A600F0EE8BF0A42CFCE435F0F8EF8AF0A42CEA
:1001B600E5F038FCE433CB8DF0A42CFCE5F03BF8FD
:1001C600EE8AF0A42CFCE5F038F8E433CF89F0A4ED
:1001D6002CFCE5F038CF3400CE89F0A42FFFE5F0F3
:1001E6003EFEE433C98DF0A42EFEE5F039CD8AF04B
:1001F600A42FFFE5F03EFEE43DFD33D0E0FB5007C3
:100206000BBB000F020370EC2CFCEF33FFEE33FE4A
:06021600ED33FD02034878
:10021C00020370EC5D046005E85904700302036688
:10022C00120331580460F6EC4860F2EC7004FDFEE9
:10023C00FF22C860DB2481C85009C39860025006B5
:10024C0002036D9850CAF582E9294B4A7005AB82BE
:10025C0002035C75F0007C1A7880C3EF9BEE9AED7C
:10026C0099400DC3EF9BFFEE9AFEED99FDE842F02D
:10027C00DC23ACF0D0E0FFD0E0FED0E0FDAB822080
:10028C00E7101BEB60BAEC2CFCEF33FFEE33FEED0A
:10029C0033FD020348E803F830E705C0F075F000C1
:1002AC00EF2FFFEE33FEED33FD40B830E7C280AAEE
:1002BC0075F020800E75F010800575F0087D007EBD
:1002CC00007F003392D530D5031203FBEC33401082
:1002DC00EF33FFEE33FEED33FDEC33FCD5F0ED22C6
:0E02EC00E5F0247EA2D513CC92E7CDCEFF2202
:1002FA00EDD2E7CD33EC3392D524814006E4FFFEFC
:10030A00FDFC22FCE4CFCECDCC24E0501174FF805A
:10031A00EDC3CC13CCCD13CDCE13CECF13CF0470F7
:07032A00F030D5DE0203FBF9
:10033100E9D2E7C933E833F892D5EDD2E7CD33EC12
:0703410033FC5002B2D5228B
:10034800EC30E7100FBF000C0EBE00080DBD000416
:100358000BEB6014A2D5EB13FCED92E7FD2274FFC2
:10036800FCFDFEFF22E480F8A2D574FF13FC7D801B
:03037800E480EF2F
:0300000002076094
:0C076000787FE4F6D8FD7581520207A7EF
:10037B00BB010689828A83E0225002E722BBFE0280
:09038B00E32289828A83E49322B3
:10039400EF8DF0A4A8F0CF8CF0A428CE8DF0A42E7D
:0203A400FE2237
:1003A600BC000BBE0029EF8DF084FFADF022E4CC3B
:1003B600F875F008EF2FFFEE33FEEC33FCEE9DEC04
:1003C600984005FCEE9DFE0FD5F0E9E4CEFD22ED4A
:1003D600F8F5F0EE8420D21CFEADF075F008EF2F94
:1003E600FFED33FD4007985006D5F0F222C398FD85
:0503F6000FD5F0EA2222
:0E03FB00C3E49FFFE49EFEE49DFDE49CFC2213
:10076C00020853E493A3F8E493A34003F68001F248
:10077C0008DFF48029E493A3F85407240CC8C3338E
:10078C00C4540F4420C8834004F456800146F6DF5D
:10079C00E4800B01020408102040809008A9E47E3C
:1007AC00019360BCA3FF543F30E509541FFEE49352
:1007BC00A360010ECF54C025E060A840B8E493A319
:1007CC00FAE493A3F8E493A3C8C582C8CAC583CA44
:1007DC00F0A3C8C582C8CAC583CADFE9DEE780BEFC
:0108F6000001
:00000001FF
